S02B0000433A2F576F726B2F736F6674776172652F4F70656E424C542F5461726765742F44656D6F2F41524DEF
S113000070070020F1000000851300008513000034
S1130010851300008513000085130000851300007C
S1130020851300008513000085130000851300006C
S1130030851300008513000085130000851300005C
S1130040851300008513000085130000851300004C
S1130050851300008513000085130000851300003C
S1130060851300008513000085130000851300002C
S1130070851300008513000085130000851300001C
S1130080851300008513000085130000851300000C
S113009085130000851300008513000085130000FC
S11300A085130000851300008513000085130000EC
S11300B085130000851300008513000085130000DC
S11300C085130000851300008513000085130000CC
S11300D085130000851300008513000085130000BC
S11300E085130000851300008513000085130000AC
S11300F072B62949072291438D4628482849294A3E
S113010000F039F828482949294A00F034F82948E8
S113011029492A4A00F02FF829482A492A4A00F096
S11301202AF82A482A492B4A00F025F82A482B495C
S11301302B4A00F020F82B482B49002200F026F827
S11301402A482B49091A082903DB002202600430DB
S113015001601C481C49884205D00268043003B47D
S1130160904703BCF7E700208646EC4600200021B8
S1130170204A9047FEE7884207D0521A05D00378F8
S113018001300B700131013AF9D17047884202D035
S113019002700130FAE7704770070020BC220000AB
S11301A00000002001000020F8010000F801000018
S11301B08C1D0000BC220000000000200000002074
S11301C08C1D00008C1D00008C1D00008C1D000087
S11301D08C1D00008C1D00008C1D00008C1D000077
S11301E0BB22000004000020F0040020F0040020E2
S10B01F0700500204513000016
S11301F8A0F58013591E012940F28680434A904293
S113020800F0828002F5807398427DD003F5007176
S1130218884279D03E4A904276D002F5807398425B
S113022872D003F5007188426ED001F57052904285
S11302386AD002F11023984266D03649884263D0C6
S11302484A1C904260D0931C98425DD0191D884284
S11302585AD00831884257D01031884254D02031BE
S1130268884251D0403188424ED0803188424BD0A8
S1130278402849D0B0F1102F46D0274A904243D0A5
S113028802F57D2398423FD0244988423CD0244A31
S1130298904239D0703A904236D0B0F1101F33D022
S11302A8204B984230D003F5807188422CD0A1F5B8
S11302B8F872904228D01032904225D002F10053AF
S11302C8984221D0184988421ED04A1C90421BD01B
S11302D8931C984218D0191D884215D0134A90428D
S11302E812D0531C98420FD0991C88420CD0B0F1FC
S11302F8202F09D00E4A904206D0082804D00D4B6E
S1130308C11A484248417047012070470001100053
S1130318000110100100002000400010000110200E
S113032880000030000100100100101001000010CE
S1130338010010200010100010B50446FFF758FF04
S113034820B909484FF4FC7101F02EFB220FA1B229
S1130358C4F3044401FA04F4044B53F82200026879
S11303681443046010BD00BFE81D0000541E0000C3
S113037801387FF4FDAF7047464B70B51A680446E0
S113038812F0E04F05D0186843490140B1F1805F8D
S113039801D1002C7DDB4148414903680E6823F4F0
S11303A8800545F4006546F4006205600A60990713
S11303B801D5A00703D5D90719D5E30717D464F0E5
S11303C80300364B0540002A1D6005DA06F070026A
S11303D8302A05D0702A02E005F03001302902D114
S11303E84FF4805001E04FF40020FFF7C1FF2D4B7C
S11303F82D49334025F45F5543F2F07043F4006609
S113040820402140294A25F03005054304F008031B
S113041846EA010022494026166050EAC30602F162
S113042808024BBF0E60156015600E601020FFF7C0
S11304389FFF1F4A25F0F86020F00303224013436E
S113044804F0FC5126F0FC52600042EA010207D590
S1130458184822F48002204043F48003024301E058
S113046822F0804221050BD44FF400411248006861
S1130478400601D40139F9D123F4006322F400625F
S113048806480749036010200A60BDE87040FFF77A
S11304986FBF70BD00E00F400000FF7060E00F40C8
S11304A870E00F408FDFFF7F3020008058E00F405E
S11304B80300C0070000404050E00F405F4B70B598
S11304C81A6810331B68002BB4BF03F0700102F0E4
S11304D83001202937D004D869B1102940F0AB8005
S11304E80FE0602954D070294FD0302940F0A38000
S11304F847F2305056E05249C2F3841051F82000B4
S113050850E05049086810F0E04F44D00C684E4859
S11305182040B0F1805F3ED00C684B4820404B4CE3
S1130528A04203D1096888B2022836D04548464912
S113053804682140464CA14201D0464832E0006894
S113054881B251B3F9E73F49086810F0E04F26D06B
S11305580C683D482040B0F1805F20D00C683A48D0
S113056820403A4CA04203D1096888B2022818D026
S11305783448354904682140354CA14201D03648F5
S113058810E0006881B261B1F9E74FF4004009E076
S11305984FF4800006E0314804E0314802E0314875
S11305A800E03148002B02DA13F4006F01E012F482
S11305B8006F28D12D4D2968224D2C6814F0E04F86
S11305C843F6E07404EA01044FEA541405D02E6893
S11305D81D4D3540B5F1805F05D1023401F01F058A
S11305E86043023504E0604301F01F0501356D00E6
S11305F8B0FBF5F011F4804F18BF4008090448BF58
S1130608800842F48002510216D5002B0DDA5900F5
S113061805D51A0503D44000C3F3865201E0C3F399
S1130628C552531CB0FBF3F070BDC2F3C353591C3D
S1130638B0FBF1F070BD002070BD00BF60E00F405A
S11306488C1D000000E00F400000FF700000011046
S1130658000003100024F40000093D00C0E1E40098
S1130668001BB70070383900C0C62D0064E00F4085
S1130678462810B5044605D91A484FF4D57101F037
S113068893F90EE0042804D1174B186840F480301D
S113069805E0052805D1144B1A6842F400301860A7
S11306A810BD062C04D1104B196841F48020F6E7DC
S11306B80F2C04D10D4B1A6842F00200EFE7A4F1A5
S11306C810031F2B05D8012000FA03F308490B6017
S11306D810BD2F2C05D9303C012101FA04F4054A38
S11306E8146010BD601E000024ED00E010E000E07E
S11306F800E100E004E100E0462810B5044605D90D
S11307081A484FF4F77101F04FF90EE0042804D1A8
S1130718174B186820F4803005E0052805D1144BE0
S11307281A6822F40030186010BD062C04D1104B4E
S1130738196821F48020F6E70F2C04D10D4B1A68B0
S113074822F00200EFE7A4F110031F2B05D80120C3
S113075800FA03F308490B6010BD2F2C05D9303C6F
S1130768012101FA04F4054A146010BD601E00005A
S113077824ED00E010E000E080E100E084E100E026
S1130788B0F1402F44D0234B984241D0A3F5A62181
S113079888423DD001F5A822904239D0A2F5A6237B
S11307A8984235D003F5A821884231D0A1F5A62274
S11307B890422DD002F5A823984229D0A3F55C31A4
S11307C8884225D001F56032904221D0A2F55C33ED
S11307D898421DD003F56031884219D0A1F55C32E6
S11307E8904215D002F56033984211D0A3F55C31DC
S11307F888420DD001F56032904209D0A2F5083341
S1130808984205D003F50C31421A504250417047C2
S1130818012070470080054070B504460D46164611
S1130828FFF7AEFF18B91048E42101F0BDF8022E15
S113083803D90D48E62101F0B7F8D4F8003416F0CE
S1130848010F14BF2B43AB4304F580621360D4F843
S1130858200416F0020F04F5846114BF054320EA4E
S113086805050D6070BD00BFCE1E0000F8B5044636
S11308780D4617461E46FFF783FF20B93E484FF43E
S1130888DD7101F091F87B1E012B08D9042F06D0E5
S11308980C2F04D038484FF4DF7101F085F8082E86
S11308A80FD00A2E0DD00C2E0BD0092E09D00B2EEA
S11308B807D00D2E05D026B12F4840F2C51101F0FE
S11308C873F8D4F8000517F0010F14BF2843A843A0
S11308D804F5A0621060D4F8041517F0020F14BFD1
S11308E82943A94304F204531960D4F8080517F0FE
S11308F8040F14BF2843A84304F5A1621060D4F878
S1130908181517F0080F14BF2943A94304F5A36366
S11309181960D4F80C0516F0010F14BF2843A84336
S113092804F20C521060D4F8101516F0020F14BF1C
S11309382943A94304F5A2631960D4F8140516F0F1
S1130948040F14BF2843A84304F214521060D4F8C7
S11309581C1516F0080F04F21C5314BF2943A943AD
S1130968196004F5A560D4F828250EB9154301E0EB
S113097822EA05050560F8BDCE1E000070B50546DF
S11309880C46FFF7FDFE20B908484FF4647101F0E6
S11309980BF8284621460222FFF73EFF2846214647
S11309A804220823BDE87040FFF760BFCE1E000094
S11309B870B505460C46FFF7E3FE20B9084840F237
S11309C81F5100F0F1FF284621460222FFF724FFB9
S11309D82846214601220823BDE87040FFF746BF98
S11309E8CE1E0000830510B5044603D00C488421AC
S11309F800F0DAFF0B4B01221A600B4843F8144C41
S1130A08143B0833186019688A07FCD4074A13682A
S1130A1813F0010F14BF4FF0FF30002010BD00BFCA
S1130A28371F000014D00F40020042A40CD00F401E
S1130A3870B50C46A1070646154603D02548C821BB
S1130A4800F0B2FFAA0703D02248C92100F0ACFF86
S1130A58214B012221481A600168CB0719D4234687
S1130A682BE075B11E4A043D881853F8041B016035
S1130A78A01B1A1812F07C01F3D11A480068002848
S1130A88EFD0194C194E26602168C807FCD41446C7
S1130A981E462DB1164B24F07F021A603346E7E751
S1130AA81448016811F0010F14BF4FF0FF30002003
S1130AB870BD0268D107FCD404332A199A42EFD0D6
S1130AC80B48311B0360C8580B4A08491060101DB5
S1130AD80160EEE7371F000014D00F40A0E10F407B
S1130AE800D10F4030D00F4020D00F40010042A465
S1130AF800D00F400CD00F4004D00F40074B984251
S1130B0809D003F58051884205D001F58052831A33
S1130B185842584170470120704700BF00C0004048
S1130B2810B50446FFF7EAFF20B908484FF4CF711F
S1130B3800F03AFFE36A43F01000E062216B41F4ED
S1130B48407242F00103236310BD00BFA41F0000DC
S1130B5810B50446FFF7D2FF20B909484FF4DF71F6
S1130B6800F022FFA3691907FCD4E06A20F0100101
S1130B78E162226B22F4407323F00100206310BD6C
S1130B88A41F0000F8B504460E4615461F46FFF795
S1130B98B5FF20B92A4840F20D1100F005FF25B928
S1130BA827484FF4877100F0FFFE264A136813F0B4
S1130BB8E04F1CD0116824480840B0F1805F16D07B
S1130BC81368214921481940814203D1126893B21C
S1130BD8022B0CD01B481C4A01681D4B0A409A4240
S1130BE801D0082204E0006881B20029F9D110225A
S1130BF86A43964204D2124840F20F1100F0D4FE20
S1130C082046FFF7A5FFB6EB051F236B04D243F07C
S1130C18200121636D0802E023F020002063F60020
S1130C28B6FBF5F56A1C0020D309C2F345056362D7
S1130C38A562E762A0612046BDE8F840FFF770BFEF
S1130C48A41F000000E00F400000FF700000011026
S1130C580000031010B50446FFF750FF20B90548FB
S1130C6840F2E93100F0A0FEA06980F02001C1F350
S1130C78401010BDA41F000010B50446FFF73EFF46
S1130C8820B9064840F2094100F08EFEA369D8064F
S1130C9854BF20684FF0FF3010BD00BFA41F0000F0
S1130CA838B504460D46FFF729FF20B9064840F237
S1130CB85B4100F079FEA3699A0602D425600120FD
S1130CC838BD002038BD00BFA41F0000074B984260
S1130CD809D003F58051884205D001F58052831A62
S1130CE85842584170470120704700BF0000044033
S1130CF8094B98420DD003F58051884207D0A1F5DD
S1130D08005290420CBF37204FF0FF307047392013
S1130D1870473820704700BF00100440016082B05B
S1130D2800210191019B042B02DC0198411CF8E786
S1130D3802B0704773B5054620F47F6020F00F00B9
S1130D48FFF7D6FF421C044603D11048F92100F0EE
S1130D582BFE0121A4F1300201FA02F00C4B1E68AB
S1130D68064002D02046FFF7C7FC2B6800210191FA
S1130D78019B042B02DC019A511CF8E72D6816B17B
S1130D882046FFF775FC28467CBD00BF10200000F4
S1130D9804E100E0F8B50446FFF798FF20B92248BB
S1130DA840F2D91100F000FE20460121FFF7B6FFFA
S1130DB804F120052846FFF7BDFF10F40046F7D1DB
S1130DC804F124073846B021FFF7A8FF314604F19F
S1130DD83400FFF7A3FF314604F13800FFF79EFF04
S1130DE801262846FFF7A6FF0004FAD43146284610
S1130DF80136FFF793FF212EF3D138460C21FFF774
S1130E088DFF01262846FFF795FF0104FAD43146E1
S1130E1828460136FFF782FF212EF3D1201DBDE8B5
S1130E28F840FFF787BF00BF1020000010B5044644
S1130E38FFF74CFF20B9074840F23A2100F0B4FD0F
S1130E482046FFF777FF20F001012046BDE8104057
S1130E58FFF764BF1020000070B505460C46FFF785
S1130E6835FF20B932484FF4597100F09DFD24B97B
S1130E782F4840F2653100F097FD2368981E0E282C
S1130E8804D92B4840F26B3100F08EFD61684A1E8C
S1130E98072A04D926484FF45C7100F085FDA6683A
S1130EA8731E032B04D9224840F2753100F07CFDEF
S1130EB8E068411EB1F5806F04D31D4840F27B31D0
S1130EC800F072FD2846FFF735FF064646F041015B
S1130ED82846FFF723FF6268531E22681803531E2F
S1130EE800F4E0411802E36800F47062581EA36835
S1130EF8114300F03F02581E11438201D3B2194333
S1130F0805F10C00FFF70AFFE16805F118004A1E15
S1130F18C2F38311FFF702FFF30754BF26F0400121
S1130F2826F041012846BDE87040FFF7F7BE00BF30
S1130F381020000038B504460D46FFF7C7FE20B957
S1130F481A4840F2925100F02FFD032D2AD8DFE809
S1130F5805F0020D151D04342046FFF7EBFE6FF073
S1130F681F0105462046FFF7D9FE1CE004F58070F2
S1130F78FFF7E0FE054604F582700EE004F5907074
S1130F88FFF7D8FE054604F5927006E004F5B07044
S1130F98FFF7D0FE054604F5B270FFF7CBFE45EA2D
S1130FA8004500E00025284638BD00BF1020000099
S1130FB82DE9F04F87B005468B4617461C46FFF7C8
S1130FC885FE20B9714840F25F6100F0EDFC0BF139
S1130FD8FF331F2B04D96D484FF4CC6100F0E4FCB7
S1130FE8042C04D9694840F2666100F0DDFC05F17F
S1130FF8200A5046FFF79EFE0304F8D4D7F800C031
S1131008BCF5006F3ABFBA68C2F380020122042C0F
S113101800F2B880DFE804F0031E070A1600012175
S11310284FF4807311E000210B4616E000214FF4C1
S113103880534FF4005E41F6FF744FF6FF764FF08D
S1131048D3080FE001214FF4905300244FF4005EBD
S1131058264605E000214FF480738E460C460E4662
S11310684FF09308B86810F0080F08D07C681AB1DC
S1131078A6B2C4F30C4402E06605F40C164600F06C
S11310882809B9F1280F00F0180908BF44F40044EE
S1131098B9F1180F08BF44F4804410F0380F18BF92
S11310A84FF0D30848F0200818BF43F48053CDF814
S11310B814804AB11FFA8CF2CCF30C49049249F417
S11310C840424EEA020906E04FEA4C5C4EEADC4E26
S11310D84EF400490492FA6802F00F0843EA08083B
S11310E883055CBF48F080031FFA83F8C30748BF31
S11310F848F40068800748BF48F4806829BB05F1B4
S113110824000599FFF70AFE05F128003146FFF788
S113111805FE05F12C002146FFF700FE05F130001D
S11311280499FFF7FBFD05F134004946FFF7F6FD86
S113113805F138004146FFF7F1FD50460BF03F0139
S113114807B0BDE8F04FFFF7E9BD3B6905F13C0C7A
S113115800209042D3DA471C9742195C03DADF5D1A
S113116841EA0721871C60460CF1040C03920293A0
S1131178CDF804C0FFF7D2FD3846DDF804C0029B61
S1131188039AE6E707B0BDE8F08F00BF102000001F
S11311982DE9F74F0546894614461E46FFF796FD86
S11311A820B9654840F2C17100F0FEFB09F1FF3334
S11311B81F2B04D9604840F2C27100F0F5FB05F119
S11311C884084046002E14BF7B21732105F1800753
S11311D809F03F09FFF7A2FD38464946FFF79EFD8F
S11311E83846FFF7A7FD0004FAD405F18800FFF795
S11311F8A1FD834605F18C00FFF79CFD824605F1AD
S11312089000FFF797FD024605F194000192FFF75D
S113121891FD064605F19800FFF78CFD10F4807FD8
S113122806F40051019A02D119B9002302E00029F9
S1131238FBD14023A36016F480434FEAC64608D086
S113124891B2A26841EAD60642F004012660A16080
S113125801E0760D2660410403D5A26842F480714A
S1131268A160C20426D54FEACA42D10C3BB11FFA89
S11312788BFB4BEA014363606FF0604203E08B1021
S1131288636040F2FF72934202D1A168490603D415
S1131298A36843F00802A2601AF4004F03D0A168BF
S11312A841F02803A3601AF4804F03D0A26842F0E7
S11312B81801A160020503D5A36843F00102A260E6
S11312C8430503D5A16841F00203A36001042ED5A8
S11312D8A66800F00F0A16F04006C4F80CA008D05F
S11312E840460421FFF71AFD38464946FFF716FD24
S11312F813E0D4F810B09C355645F1DA2846FFF7C8
S113130819FD721C043552450BF8060003DA030A6A
S11313180BF80230B21C1646EEE73846FFF70AFD12
S11313280204FAD4A26842F08001A16001E000201E
S1131338E060BDE8FE8F00BF1020000008B50B4830
S1131348FFF71AF80A48FEF7F7FF03214FF0402089
S1131358FFF72EFB0748FEF7EFFF07480321FFF7C7
S11313680DFB00F059FB00F064FBFCE78003C001AF
S113137801000020080000200070004001483D21C1
S113138800F012BB7B20000008B500F0C8F978B162
S113139800F088FB00F0DEF900F0B8F9054B20F006
S11313A8604020F07F01196000F0B0F9426890476E
S11313B808BD00BF08ED00E0F8B505460E4617461F
S11313C80024A3B29F4205D0A05D605500F0A7FB9E
S11313D80134F6E7F8BDFEF787BE000070B50024B7
S11313E80646254600F09BFB094BE258964209D372
S11313F8191948681218964204D20C2101FB0535C4
S1131408287A70BD0C340135C02CEBD1FF2070BD97
S1131418002100002DE9F34105460068FFF7DEFFCF
S1131428FF2801D100201AE000242B1958682F68DE
S113143802AE46F8040D04EB070800F070FB3046D2
S113144841460422FFF7F4FA0028EBD1E259019946
S11314588A42E7D10434B4F5007FE6D10120BDE81F
S1131468FC81000038B5104B044698420D4606D05E
S1131478B1F5004F05D0FFF7CDFF18B910E00B4CBC
S113148800E01C46EB050BD12068A84209D0204691
S113149840F8045B29464FF40072FFF78DFF00E023
S11314A80024204638BD00BF0400002008020020A4
S11314B82DE9F8439946036821F4FF75013304467E
S11314C80E46904625F0010506D140F8045B2946EE
S11314D84FF40072FFF770FF2068A84208D0204636
S11314E82946FFF7BFFF044610B90020BDE8F8837A
S11314F821684746761AA219161D00F010FB231D11
S1131508F01AB0F5007F08D3204605F50071FFF7FF
S1131518A9FF04460028E8D0061D17F8011B08EBAC
S11315280902974206F8011BE7D10120BDE8F883B8
S1131538034A04484FF0FF3313600360704700BF49
S1131548080200200400002070B504460D46164623
S1131558FFF744FFFF2815D0601E4019FFF73EFF30
S1131568FF280FD024F4FF7323F00101B1F5004FD5
S11315780CBF05480548214632462B46BDE8704055
S1131588FFF796BF002070BD040000200802002069
S1131598F8B505460E46FFF721FF0446681E801974
S11315A8FFF71CFFFF2C05464DD0FF284BD0844283
S11315B849D8032C47D9132845D8002600F0AFFA98
S11315C8224B0C2202FB06310F7AA74201D10C6888
S11315D804E00136102EF1D14FF0FF34002700F05B
S11315E89EFA1A4A0C2000FB0723197AA94201D152
S11315F81F6804E00137102FF1D14FF0FF370026A0
S113160800F08DFA114A0C2000FB0623197AA9422E
S113161801D15D6803E00136102EF1D100253F1B8E
S11316287819C0F38F270025BD420AD200F077FA53
S11316382046FFF7D7F904F5806420B96A1C95B2EF
S1131648F2E70120F8BD0020F8BD00BF002100002A
S11316580E4B07B51A68013216D058689968DA68CB
S11316680918881819695A69401881189869DB6932
S11316780A18D118484202AA42F8040D042148F273
S1131688F000FFF761FF00E001200EBD0400002018
S113169848F204034FF400410A68186848F2080342
S11316A819688018421848F20C000368D11848F2E7
S11316B81002106848F214031A680918881848F2C6
S11316C818010B68C21848F2F00001685318D3F1E6
S11316D8010038BF002070470A4808B50368013381
S11316E805D1094801684B1C06D1012008BDFFF744
S11316F891FE0028F5D108BDFFF78CFE003018BF15
S1131708012008BD04000020080200204FF4004016
S11317187047FFF70DBFFFF717BFFFF739BFFFF794
S1131728B7BF08B5FFF794FF18B1BDE80840FFF745
S1131738D3BF08BD054B00224CF24F3105201A6077
S113174859609A601860024B1A60704710E000E014
S11317580C040020014B00221A60704710E000E0DE
S1131768044B1868C30303D503490A68531C0B6068
S1131778704700BF10E000E00C04002008B5FFF734
S1131788EFFF014B186808BD0C04002010B507488A
S1131798FEF7D2FDFEF792FE014605484FF461427A
S11317A86023BDE81040FFF7EDB900BF0100001049
S11317B800C00040402970B506460D4603D91648B6
S11317C8572100F0F1F815482946FFF769FA30B1B6
S11317D81248FFF73FFA30B900F0A1F9F8E70E48CC
S11317E85B2100F0E1F80024A3B2AB4213D200F06D
S11317F896F90A48315DFFF753FA30B10748FFF705
S113180829FA30B900F08BF9F8E70348642100F0AD
S1131818CBF80134E8E770BDC021000000C00040E7
S1131828F8B5154C064625786DB91448FFF724FA1F
S1131838421C01D10020F8BD1149124B0870012047
S113184820701D70F6E70F4D0C482F78FFF714FA37
S11318580137431CEED00A492B78C8550A78581C1E
S1131868C3B29A422B70E5D130460131FFF7A4FD8B
S1131878002222700120F8BD1104002000C000409D
S1131888120400201004002010B524488AB0FEF782
S113189853FD2348FFF77EFA042310220393019291
S11318A840F2A4600823EBB1511CC918B0FBF1F451
S11318B8413CE4B20A2C13D81024B4FBF1F44C4391
S11318C8102C0DD1032B019298BF03931022B2FB65
S11318D8F1F0049001A912480293FFF7BDFA08E059
S11318E8013BE0E76438013ADCD10E48902100F06E
S11318F85BF80B48FFF79AFA40F26761082201F592
S1131908CC7305910693079208920548012105AA0C
S11319180223FFF74DFB0AB010BD00BF0001100001
S1131928000004403722000030B5044687B00D4655
S113193810480121FFF7FEFA820703D50E48AB21B0
S113194800F032F840F2E17301930A4800230221BF
S113195801AA039304950594FFF72AFB012105487E
S1131968FFF7E8FA044600F0DAF8A307F6D407B05C
S113197830BD00BF000004403722000010B502212A
S113198886B004460748FFF7D5FA10F0010007D0DF
S11319980121044801AA0B460594FFF7F9FB01202D
S11319A806B010BD0000044008B5034B1860034896
S11319B8016000F0B4F8FCE7540400205804002047
S11319C810B500F0A9F8012811D0094C2378012B8F
S11319D80DD1FFF7D3FE07490A6802F5FA73984256
S11319E805D300202070BDE81040FFF7CDBC10BD22
S11319F85C0400206004002008B5054B01221A701D
S1131A08FFF7BCFE03490860BDE80840FFF7D8BFEC
S1131A185C0400206004002008B500F07FF8FFF79C
S1131A2889FEFFF776FE00F00FF8BDE80840FFF7DF
S1131A38E3BF08B500F073F8FFF792FE00F014F85E
S1131A48BDE80840FFF7BCBF10B5064C00F072F8BB
S1131A58FFF71AFF01232370FFF798FE0020207078
S1131A6810BD00BF0000002008B50C48FFF786FF32
S1131A78012804D10A4B1870084800F079F807487F
S1131A88FFF7CEFE012807D105480022027003485B
S1131A98BDE8084000F06CB808BD00BF640400202D
S1131AA800000020704700000A4B70B51A780646FB
S1131AB8012A0C461D4602D1C9B2FFF735FF287822
S1131AC818B93046E1B2FFF775FEBDE8704000F082
S1131AD847B800BF00000020054B1878411ECBB260
S1131AE8022B02D8034AD05C70474020704700BFDD
S1131AF800000020AD220000054B1878411ECBB22F
S1131B08022B02D8034AD05C70474020704700BFBC
S1131B1800000020B022000000F01AB87047704797
S1131B28034BFE2218710220DA70A3F844007047B0
S1131B38A4040020054B00221A709A6483F84320F9
S1131B48A3F844209A705A70704700BFA404002078
S1131B58024B1878003018BF01207047A4040020F5
S1131B68024B002283F84320704700BFA4040020DE
S1131B78F8B503780546FF2B804C14D100210125C4
S1131B88E37010236170237161712570FFF7A4FF5E
S1131B98A071FFF7B1FFE071FFF7AEFF020A2272EE
S1131BA86572A5727FE02678012E40F0E580F32B5C
S1131BB855D01FD8CF2B00F0BD8006D8C92B00F014
S1131BC88380CC2B40F0BF80BBE0D12B00F0AC80ED
S1131BD8C0F08C80D22B40F0B6800025FF22E27042
S1131BE825716571FFF778FFE571A071257265723B
S1131BF8072396E0FA2B4BD00AD8F52B11D01AD329
S1131C08F62B40F0A080FF22E2704068A06495E0C3
S1131C18FD2B4AD0FE2B53D0FC2B40F0948000209F
S1131C2892E0FFF759FF6A78904201DC22208BE0AA
S1131C38201DA16C08E0FFF74FFF6B789842F5DD93
S1131C486968201DA1646A78FFF7B6FBFF21E1707B
S1131C586A78A06C1318A36469784B1C61E0FF20B0
S1131C68E070A36C6C6800201C19A34204D013F81C
S1131C78011B4218D0B2F8E7404B0022C3F8070012
S1131C880121082019715A719A71A3F844005DE082
S1131C983B4B0021FF200722E070A364217161718E
S1131CA8A171C4F8072008233BE062780021FF23D0
S1131CB8E37021716271A171E1712172062330E030
S1131CC800222270627037E0A76CFFF705FF6A1CD8
S1131CD8411E3846FFF71FFD98B3FF20A56CE0703E
S1131CE8FFF7FAFE013D2918A16427E0FFF7F4FE87
S1131CF869780138884299DDFF22E270A4F84460CB
S1131D08697819B9FFF70DFD00BB1AE01B4CAA1C32
S1131D18A06CFFF700FDA0B16878A36CC118A1649A
S1131D2814E0A4F8443011E0A06C6968FFF7F5FCEE
S1131D3810B906E0FFF74FFBFF20E070A4F84460F9
S1131D4804E0312000E02020FFF7EAFE0B4C94F871
S1131D584300012802D11020FFF7E2FEB4F8441032
S1131D68064A0BB2002B07DD012082F84300D01C81
S1131D78BDE8F840FFF798BEF8BD00BFA4040020F2
S1071D88B32200007E
S1131D8C40420F0000201C0080841E0000802500AF
S1131D9C999E36000040380000093D0000803E004A
S1131DAC00004B00404B4C0000204E00808D5B002B
S1131DBC00C05D000080700000127A0000007D00FD
S1131DCC80969800001BB7000080BB00C0E8CE00D2
S1131DDC647ADA000024F4000000FA00433A2F5726
S1131DEC6F726B2F736F6674776172652F4F7065AA
S1131DFC6E424C542F5461726765742F44656D6F39
S1131E0C2F41524D434D335F4C4D33535F454B5F24
S1131E1C4C4D3353383936325F43726F7373776F6B
S1131E2C726B732F426F6F742F6964652F2E2E2F74
S1131E3C6C69622F6472697665726C69622F73794E
S1131E4C7363746C2E63000000E10F4004E10F40D7
S1131E5C08E10F40433A2F576F726B2F736F667400
S1131E6C776172652F4F70656E424C542F546172BA
S1131E7C6765742F44656D6F2F41524D434D335F2D
S1131E8C4C4D33535F454B5F4C4D335338393632DD
S1131E9C5F43726F7373776F726B732F426F6F74D0
S1131EAC2F6964652F2E2E2F6C69622F64726976EC
S1131EBC65726C69622F696E746572727570742EBA
S1131ECC6300433A2F576F726B2F736F667477618D
S1131EDC72652F4F70656E424C542F546172676556
S1131EEC742F44656D6F2F41524D434D335F4C4DF0
S1131EFC33535F454B5F4C4D3353383936325F4364
S1131F0C726F7373776F726B732F426F6F742F6969
S1131F1C64652F2E2E2F6C69622F6472697665723C
S1131F2C6C69622F6770696F2E6300433A2F576F89
S1131F3C726B2F736F6674776172652F4F70656E59
S1131F4C424C542F5461726765742F44656D6F2F26
S1131F5C41524D434D335F4C4D33535F454B5F4CB6
S1131F6C4D3353383936325F43726F7373776F72F4
S1131F7C6B732F426F6F742F6964652F2E2E2F6C29
S1131F8C69622F6472697665726C69622F666C6122
S1131F9C73686C69622E6300433A2F576F726B2F10
S1131FAC736F6674776172652F4F70656E424C5413
S1131FBC2F5461726765742F44656D6F2F41524DB8
S1131FCC434D335F4C4D33535F454B5F4C4D335353
S1131FDC383936325F43726F7373776F726B732F4A
S1131FEC426F6F742F6964652F2E2E2F6C69622FCC
S1131FFC6472697665726C69622F756172746C694E
S113200C622E6300433A2F576F726B2F736F667493
S113201C776172652F4F70656E424C542F54617208
S113202C6765742F44656D6F2F41524D434D335F7B
S113203C4C4D33535F454B5F4C4D3353383936322B
S113204C5F43726F7373776F726B732F426F6F741E
S113205C2F6964652F2E2E2F6C69622F647269763A
S113206C65726C69622F63616E6C69622E630043E6
S113207C3A2F576F726B2F736F6674776172652F7B
S113208C4F70656E424C542F5461726765742F44C3
S113209C656D6F2F41524D434D335F4C4D33535F40
S11320AC454B5F4C4D3353383936325F43726F7343
S11320BC73776F726B732F426F6F742F6964652F14
S11320CC2E2E2F2E2E2F2E2E2F2E2E2F536F75722B
S11320DC63652F41524D434D335F4C4D33532F4366
S11320EC726F7373776F726B732F766563746F7221
S11320FC732E630000800000002000000400000028
S113210C00A00000002000000500000000C000003A
S113211C002000000600000000E000000020000089
S113212C070000000000010000200000080000006F
S113213C0020010000200000090000000040010004
S113214C002000000A0000000060010000200000D4
S113215C0B00000000800100002000000C000000B7
S113216C00A00100002000000D00000000C00100D0
S113217C002000000E00000000E001000020000020
S113218C0F0000000000020000800000100000009E
S113219C0080020000800000110000000000030019
S11321AC008000001200000000800300008000008A
S11321BC13000000433A2F576F726B2F736F6674C2
S11321CC776172652F4F70656E424C542F54617257
S11321DC6765742F44656D6F2F41524D434D335FCA
S11321EC4C4D33535F454B5F4C4D3353383936327A
S11321FC5F43726F7373776F726B732F426F6F746D
S113220C2F6964652F2E2E2F2E2E2F2E2E2F2E2E31
S113221C2F536F757263652F41524D434D335F4C91
S113222C4D33532F756172742E6300433A2F576FDD
S113223C726B2F736F6674776172652F4F70656E56
S113224C424C542F5461726765742F44656D6F2F23
S113225C41524D434D335F4C4D33535F454B5F4CB3
S113226C4D3353383936325F43726F7373776F72F1
S113227C6B732F426F6F742F6964652F2E2E2F2E64
S113228C2E2F2E2E2F2E2E2F536F757263652F41EA
S113229C524D434D335F4C4D33532F63616E2E635C
S11222AC000800000800004F70656E424C54009B
S10422BC0419
S90300F10B
